:020000040800F2
:10000000481B002081020008B33600085D35000857
:10001000B1360008911E00084941000800000000A8
:10002000000000000000000000000000B7360008DB
:100030008321000800000000B5360008653D000877
:100040009B0200089B0200089B0200089B0200081C
:100050009B0200089B0200089B0200089B0200080C
:100060009B0200089B0200089B0200089B020008FC
:100070009B0200084D2100089B0200089B0200081B
:100080009B0200089B0200089B0200089B020008DC
:100090009B0200089B0200089B0200089B020008CC
:1000A0009B0200089B0200089B0200089B020008BC
:1000B0009B0200089B0200089B0200089B020008AC
:1000C0009B0200089B0200089B0200089B0200089C
:1000D0009B0200089B0200089B020008F5400008F4
:1000E0009B0200089B0200089B0200089B0200087C
:1000F0009B0200089B0200089B0200089B0200086C
:100100009B0200089B0200089B0200089B0200085B
:100110009B0200089B0200089B0200089B0200084B
:100120009B0200089B0200089B0200089B0200083B
:1001300000F002F800F090F80AA090E8000C824469
:100140008344AAF10107DA4501D100F085F8AFF246
:10015000090EBAE80F0013F0010F18BFFB1A43F0A5
:1001600001031847084B0000284B0000103A24BF39
:1001700078C878C1FAD8520724BF30C830C144BF0C
:1001800004680C607047000000230024002500264E
:10019000103A28BF78C1FBD8520728BF30C148BFEA
:1001A0000B6070476E2900F01F82702900F0698390
:1001B000662904F0CD84652904F0CA84672904F017
:1001C000C784612904F0C68403681B0A28BF41F074
:1001D0008001692900F0CC81642900F0C98175296A
:1001E00000F0C6816F2900F0F782782900F035838E
:1001F000E92900F09182E42900F08E82F52900F0CF
:100200008B82EF2900F0F482F82900F03483036830
:10021000DB0928BF41F08001632901F06780732961
:1002200001F06C80E32901F07780F32901F07C80F4
:10023000002070471FB501F0C9F80400002000211C
:1002400004F070FC401C60600020002104F054FCAD
:10025000E0601FBD10B510BD01F08AF81146FFF730
:10026000E9FF04F0CDFB01F063F903B4FFF7F2FFFF
:1002700003BC01F0A7F9000080F308887047000074
:100280000948804709480047FEE7FEE7FEE7FEE72A
:10029000FEE7FEE7FEE7FEE7FEE7FEE70448054966
:1002A000054A064B70470000C93D000831010008AF
:1002B00048150020481B0020481700204817002040
:1002C0007CB51D4616460C00009001D02044401E0F
:1002D000074B7B442A4669460190304600F09DF961
:1002E00005461CB10020694600F0AAF928467CBDED
:1002F0007503000040EA010310B59B070FD1042AE3
:100300000DD310C808C9121F9C42F8D020BA19BAE0
:10031000884201D9012010BD4FF0FF3010BD1AB145
:10032000D30703D0521C07E0002010BD10F8013B9A
:1003300011F8014B1B1B07D110F8013B11F8014BC1
:100340001B1B01D1921EF1D1184610BD10B5431CE4
:1003500002E010F8011B71B18107FAD14FF00132B0
:1003600002C88C1A8C4314EAC211F9D0C01A0A06CA
:1003700003D0C01E10BDC01A10BD0A0401D0801EDB
:1003800010BD0902FCD0401E10BD032A40F230808F
:1003900010F0030C00F0158011F8013BBCF1020FC6
:1003A000624498BF11F801CB00F8013B38BF11F847
:1003B000013BA2F1040298BF00F801CB38BF00F85E
:1003C000013B11F0030300F02B83083AC0F00880D2
:1003D00051F8043B083A51F804CBA0E80810F5E7BF
:1003E000121D5CBF51F8043B40F8043BAFF30080A2
:1003F000D20724BF11F8013B11F801CB48BF11F817
:10040000012B24BF00F8013B00F801CB48BF00F8E6
:10041000012B70474FF000020429C0F0128010F049
:10042000030C00F01B80CCF1040CBCF1020F18BFD0
:1004300000F8012BA8BF20F8022BA1EB0C0100F063
:100440000DB85FEAC17C24BF00F8012B00F8012B36
:1004500048BF00F8012B70474FF0000200B513466B
:1004600094469646203922BFA0E80C50A0E80C50D4
:10047000B1F12001BFF4F7AF090728BFA0E80C5085
:1004800048BF0CC05DF804EB890028BF40F8042B7E
:1004900008BF704748BF20F8022B11F0804F18BFEB
:1004A00000F8012B704770477047704770B50446DD
:1004B00085690068C10601D5302600E02026C00706
:1004C00007D070BDD4E9012130469047206A401C16
:1004D00020626D1EF6D570BD70B504468569007842
:1004E000C00707D170BDD4E9012120209047206AC0
:1004F000401C20626D1EF6D570BD09684A0501D505
:1005000040B27047C905FCD500B2704709684A057A
:1005100001D5C0B27047C905FCD580B2704770B52F
:100520000C460546012A05D02878800600D5EA69E0
:10053000002302E0012305E05B1C934202D2E05C51
:100540000028F9D1A869E618C01AA861286A1844D9
:1005500028622846FFF7AAFF04E0D5E9012114F834
:10056000010B9047B442F8D32846FFF7B5FF70BDA2
:100570002DE9F0410646002410687529314616A57C
:1005800010D0FFF7BAFF002802DA404213A507E0B7
:1005900031688A0701D512A502E0490704D511A5E3
:1005A000012401E0FFF7B2FF00210A2206F124072F
:1005B00009E0B0FBF2FCB0FBF2F302FB1C003030B0
:1005C00078541846491C0028F3D123462A46304661
:1005D000BDE8F04100F09BBA000000002D000000D3
:1005E0002B0000002000000011680268006A53051B
:1005F00001D508700AE0D30501D5088006E013068E
:1006000003D5C217C1E9000200E00860012070476D
:1006100001694A1C02610878704700B58FB0CDE9C6
:1006200001310021059105497944CDE903101146B6
:10063000684600F031F90FB000BD0000E5FFFFFF94
:100640000A6802F8010B0A607047D1E900239A4258
:1006500002D2531C0B601070704700002DE9FF5F41
:1006600015468A460446DFF8AC80F8440027D8E9EE
:1006700000103E46CDE9001010E03AF816106A4628
:1006800002A800F055FE411C07D02178890603D549
:10069000E269391891420DD80744761C207880060B
:1006A00002D5E069B84205DDAE42E6DB3AF8160055
:1006B0000028E2D1A069C01BA0612046FFF7F6FE2A
:1006C000D8E90010CDE90010002017E03AF8181022
:1006D0006A4602A800F02CFEB0F1FF3F81460BD025
:1006E00000250DF1080B05E0D4E901211BF80500F8
:1006F00090476D1C4D45F7D308F10100B04280468C
:10070000E4DB206A384420622046FFF7E5FEBDE8BE
:10071000FF9F0000024500002DE9F0418046D21DF8
:1007200022F007020025D2E90002F52915A614D00F
:10073000011E72F1000106DA0023D0EB030063EB27
:10074000020211A608E0D8F800108B0701D50FA609
:1007500002E0490701D50EA601251146002408F143
:10076000240704E000F08EF930323A55641C50EA58
:100770000102F7D12B46324621464046BDE8F04102
:1007800000F0C5B9000000002D0000002B000000A3
:100790002000000030B4002100F1240408E002F041
:1007A0000705D208303542EA4372DB086554491C1C
:1007B00052EA0305F3D10468002310A2250708D5E7
:1007C00004F020040C4304D0C46901230CA2641E6D
:1007D000C46130BC00F09BB910B5044621461068D6
:1007E000FFF794FE02462046BDE810400023D1E703
:1007F000D21D22F00701D1E90023CBE70000000061
:1008000030000000F0B40D460188090502D5214CE6
:100810007C4402E01F4C7C440E34002100F124068D
:1008200008E002F00F071209E75D42EA03721B09B4
:100830007754491C52EA0307F3D1027800231207C8
:1008400004D5702D06D009B1022311342246F0BC24
:1008500000F05DB901231034F8E770B504460D4689
:1008600021461068FFF752FE024629462046BDE8A1
:1008700070400023C6E7D21D22F00703D3E900230E
:10088000C0E70368126843F0200303600823C361D4
:100890000023B7E7644300002DE9F05F8946044672
:1008A0004FF0000ADFF874B1FB44C0F820A02046E6
:1008B000E1688847002874D0252806D0D4E90121B2
:1008C0009047206A401C2062F1E700265F462046E0
:1008D000E16888472028054607DB312D05D27819C5
:1008E00010F8200C08B10643F1E7B00701D526F057
:1008F0000406C4F81CA00027C4F818A02A2D09D0AB
:10090000284603F0ECFF38B304EB8708303DC8F805
:10091000185019E059F8041B204604EB8702916136
:10092000E1688847012F054618D1E069002820DAE0
:1009300026F020061DE0D8F8180000EB800005EB3B
:1009400040003038C8F818002046E168884705465E
:1009500003F0C5FF0028EED1012F0AD02E2D08D1BB
:100960002046E16888477F1C0546022F46F0200696
:10097000C4DBA069002803DA404246F00106A0610A
:10098000F00701D026F010066C2D0BD0682D09D091
:100990004C2D39D06A2D35D0742D35D07A2D33D0E9
:1009A00016E038E0E1682F4620468847B842054601
:1009B00009D16C2F26D04FF48060E16806432046B1
:1009C0008847054604E06C2F1AD04FF48070064328
:1009D0000DB3A5F14100192802D8203546F4006670
:1009E0004A462946204626604E46FFF7DBFB80B18B
:1009F00001280BD0F61D26F0070000F1080956E784
:100A00004020E4E78020D8E70020D6E706F104097B
:100A10004DE7284652E7206ABDE8F09FF442000007
:100A200010B5203AC0F00B80B1E81850203AA0E889
:100A30001850B1E81850A0E81850BFF4F5AF5FEABD
:100A4000027C24BFB1E81850A0E8185044BF18C970
:100A500018C0BDE810405FEA827C24BF51F8043B17
:100A600040F8043B08BF7047D20728BF31F8023B6B
:100A700048BF11F8012B28BF20F8023B48BF00F8FF
:100A8000012B704730B5B0F10A024FEA900E71F1B8
:100A900000034EEA817EB0EB0E0061EB91014FEA5C
:100AA000101E4EEA017E10EB0E0041EB11114FEAD1
:100AB000102E4EEA016E10EB0E0041EB11214FEAB1
:100AC000104E4EEA014E10EB0E0041EB1141401862
:100AD00041F100014FEAD00040EA41704FEAD101F4
:100AE00010EB80054FEA810444EA907444EB010462
:100AF0006D1944EB0404521BA3414FF0000348BF9F
:100B00000A3200D530BD401C41F1000130BD2DE955
:100B1000F0470D4699469246044600F124080168C4
:100B2000880604D5E06921F01001216000E0012071
:100B3000A84201DD471B00E00027A1697A1902EBFA
:100B40000900081AA0612078C00602D42046FFF7E9
:100B5000ADFC002608E0D4E901211AF80600904710
:100B6000206A401C761C20624E45F4DB2078C006CB
:100B70000AD52046FFF79AFC06E0D4E9012130208F
:100B80009047206A401C2062381EA7F10107F4DC60
:100B900007E0D4E9012118F805009047206A401CBD
:100BA0002062281EA5F10105F3DC2046FFF794FC26
:100BB0002078000602D50220BDE8F0870120FBE77F
:100BC00070472DE9FF4F0C461E464FF0FF378BB0A4
:100BD000D2E90001DDF860800A908A46C1F30A5527
:100BE00005B93D46002108464FF00000BAF1000F5C
:100BF00000F4400005DA00EB80004FF4400101EA08
:100C000050004FEA9059B9F1010F00DDB9460A983A
:100C100050EA4A000ED044F61050A5F2FF35454385
:100C20002F14B8F1000F1ED07542291E1EDDC9F128
:100C300000021CE0B8F1010F4FF0000001D030219C
:100C400003E0F24305E02154401CB042FBDB304698
:100C50000022002121540B99C1F80880C1E900202D
:100C60000FB0BDE8F08FBD1B6D1CDEE74A4600DA11
:100C7000694206A800F0EEFB06AB93E8070003AB61
:100C800083E8070050460A9900F0A3FC8DE80700AE
:100C9000A0F500501F3800900398002D09DD42F2A6
:100CA0001F014A46084403A90390684600F002FF6A
:100CB00008E0A0F500504A461F3803A90390684693
:100CC00000F00CFF8DE807000004000C03D04FF08B
:100CD000FF30410800E01046B8F1000F03D00022B9
:100CE000009215461EE0751E05D4FFF7CBFE30328C
:100CF00062556D1EF9D5B3460122084302D0002289
:100D00007F1C04E02078302801D100227F1E002AB9
:100D1000099786D01DE0112D07DAFFF7B3FE3032B8
:100D200062556D1C50EA0102F5D1084302D00098CB
:100D3000C8B10EE00021681E05E0235C625C6354CC
:100D40002254401E491C8142F7DBAB46A81B401EC3
:100D50000990002004F80B000B98099AC0F808804D
:100D6000C0E9002B7CE711264FF0000859E72DE978
:100D7000F04F88460446D21D22F0070191B0D1E918
:100D80000001CDE90A0103F079FD02460B98C00F7E
:100D900001D02D2007E02068810701D52B2002E03B
:100DA000202101EAC000032A099001D0072A05DBAF
:100DB00003464146204600F00DFB0BE120788006FB
:100DC00001D5E06900E00620B8F1650F814606D044
:100DD000B8F1660F18D0B8F1670F70D131E000207C
:100DE000B9F1110F009001DB112301E009F10103BA
:100DF0000AAA01A90CA8FFF7E4FEDDE90C700026A1
:100E000009F10105834647E001204B4600904FF071
:100E100000470AAA01A90CA8FFF7D3FEDDE90DB02F
:100E20000C995D46002610B909F101000D18B9EBC7
:100E3000050003D4C0F1FF3609F10105A5EB090057
:100E40002BE0B9F1010F01DA4FF001090020B9F1EF
:100E5000110F0090484601DD112300E003460AAA65
:100E600001A90CA8FFF7ADFEDDE90C704D46002688
:100E70008346207800070AD4AB4500DA5D4601A816
:100E8000012D04DD411911F8011C302907D04F450F
:100E900002DA17F1040F04DA012082460FE06D1E1A
:100EA000EEE7002F02DCED1B3E4403E0781CA84275
:100EB00000DD7D1CB81B00F1010A4FF000472078CF
:100EC000000703D4AA4501DB4FF0FF3A0021B7F138
:100ED000004F0DF143088DF8431024D002202B233E
:100EE000002F01DA7F422D230A21021EA0F101000A
:100EF00000DC5FB197FBF1FC97FBF1F201FB1C7C7E
:100F000017460CF1300C08F801CDEEE7A8F101000E
:100F100003702188090501D5452100E06521A0F174
:100F2000010800F8011C09980FA9A1EB0807FF1D93
:100F300000B10120411901EBEA70A1693844081A97
:100F4000401EA0612078C00602D42046FFF7AEFA0A
:100F5000099828B1D4E901219047206A401C2062F9
:100F60002078C00622D52046FFF7A0FA1EE0002E0A
:100F700004DBB34502DD01A8805D00E03020D4E948
:100F800001219047206A401C2062761CAAF10100D2
:100F90005FEA000A0AD100F019FAC0680168405CF3
:100FA000D4E901219047206A401C2062281EA5F147
:100FB0000105DCDC07E0D4E9012118F8010B9047BA
:100FC000206A401C2062381EA7F10107F3DC20468E
:100FD000FFF782FA032011B043E600002DE9F04F3D
:100FE00004460D46D21D22F0070089B0D0E90092D8
:100FF00048461746394603F041FC0246F80F01D037
:101000002D2307E02068810701D52B2302E0202152
:1010100001EAC0038DF820300BB1012000E0002070
:10102000032A824601D0072A04DB2946204600F025
:10103000D1F93DE12078800601D40D2500E0E56975
:10104000C7F30A560D2D49DA00214FEA175B08460F
:101050004FF00000002F00F4400007DA00EB8000A2
:101060004FF4400100EBD07001EA600081150129C6
:1010700001DD4FF0FF3100224FEA850CBCF1180F63
:1010800006D31346ACF118004FF08052C24003E083
:101090004FF4801323FA0CF30CF10C0CBCF1200F6D
:1010A00004D3ACF1200C09FA0CF001E007FA0CF0C3
:1010B00000294FF0004801DD18B90FE00ED140457E
:1010C0000CD319EB02095F4121B9404502D19F437E
:1010D00029EA0209BBEB175F00D0761C20880005C7
:1010E00002D57B48784402E079487844193808AA48
:1010F000302302F80A30037C0AF10101002E0AF1C4
:10110000020A53546A4602DC4FF0300101E04FF00E
:1011100031014FF001088DF8001002D0A6F2FF3621
:1011200003E059EA470100D06A4E002D02DC217825
:10113000090704D54FF002082E218DF80110C4468E
:1011400000210BE0C7F303433F01C35C491C6D1E44
:1011500002F80830052908F1010801DA002DF1DC58
:1011600000210CE000EB1973491C1B786D1E082947
:1011700002F808304FEA091908F1010801DA002DD8
:10118000F0DC2178890602D514E0A8F10108E045D9
:1011900005DD02EB080111F8011C3029F5D0B8F18A
:1011A000000F07DD02EB080111F8011C2E2901D107
:1011B000A8F10108002D05DD3E2102F808106D1E82
:1011C00008F10108407C002E02F8080008F101082F
:1011D00004DA2D20764202F8080002E02B2002F803
:1011E00008000A214FF47A70864208F101080BDBEF
:1011F00096FBF0F3303302F8083096FBF0F308F179
:10120000010800FB136601E0642E0CDB642096FBF2
:10121000F0F3303302F8083096FBF0F308F10108E0
:1012200000FB136601E00A2E06DB96FBF1F030307E
:1012300002F8080008F1010896FBF1F001FB1060CC
:10124000303002F80800A16908F1010808EB050236
:1012500002EB0A00081AA0612078C00602D42046DA
:10126000FFF724F9216A08AE01EB0A00206204E0CE
:10127000D4E9012116F8010B9047BAF1010AF7D21F
:101280002078C00602D52046FFF710F96E4609E027
:1012900016F8010B3E280FD0D4E901219047206AAF
:1012A000401C2062B8F10108F2D22046FFF714F981
:1012B00009B00320BDE8F08F206A2844206203E0D3
:1012C000D4E90121302090476D1EEBD3F8E70000F0
:1012D000DC3A000002FCFFFF10B5436913B1AFF325
:1012E000008001E0FFF71BF9012010BD127800F12A
:1012F00024010A7000224A700122EDE711684FF0C4
:10130000FF32E9E710B5436913B1AFF3008001E0A4
:10131000FFF7A4F9012010BD128800F12401828496
:101320000022C2840122EDE711684FF0FF32E9E7A5
:1013300070B516460C46054600F040F8036893F871
:101340000101012806D0FF2C0FD8185D68B10120DB
:101350002C7070BDD3F807013246214603F2071303
:1013600003442846BDE8704018474FF0FF3070BD79
:10137000754600F0E3F8AE4605006946534620F096
:101380000700854618B020B5FEF788FFBDE820406D
:101390004FF000064FF000074FF000084FF0000B31
:1013A00021F00701AC46ACE8C009ACE8C009ACE8E4
:1013B000C009ACE8C0098D467047000010B500F0C8
:1013C00005F8001D10BD00BF5D37000000487047E4
:1013D000081500202DE9F0411F4604460326016848
:1013E000072A01F4006004DB08B116A505E016A584
:1013F00003E008B115A500E015A521F0100020605C
:10140000A069C01EA0610FB1401EA0612046FFF779
:101410004DF84FB1D4E9012138469047206A401C6D
:101420002062C01C206206E0206AFAE7D4E90121AC
:1014300015F8010B9047761EF8D22046FFF74CF8BE
:10144000BDE8F0814E414E006E616E00494E46008F
:10145000696E66002DE9F047814616468AB033482A
:1014600078440DC88DE80D0030487844801C03ACEA
:101470000DC884E80D0041F69B300844372190FBED
:10148000F1F290FBF1F5A5F1800501FB12041B3C84
:1014900002D56442012000E00020DFF890A08046E1
:1014A0000027FA44AAF1BE0A0DE0E00709D032464F
:1014B000684607EB47010AEB810100F00FFB8DE85E
:1014C000070064107F1C002CEFD1184F7F44AC3F05
:1014D00018E0E80714D007EB04100DF1180A90E8A3
:1014E0000E008AE80E00C068F04201D198190890F9
:1014F000324606A903A800F0F1FA03AB83E807001F
:101500006D10641C002DE4D132466946B8F1000F1D
:1015100003A802D000F0CEFA01E000F0DFFAC9E93A
:101520000001C9F808200AB0BDE8F087F0370000D4
:101530000446AFF300802046FEF797FE0048704750
:10154000E81400204FF0013C50F8042B51F8043B04
:101550009A4221D1A2EB0C03934313EACC1317D187
:1015600050F8042B51F8043B9A4215D1A2EB0C031E
:10157000934313EACC130BD150F8042B51F8043BDE
:101580009A4209D1A2EB0C03934313EACC13DBD0AC
:101590004FF00000704700BFD01A01BAB1FA81F1D4
:1015A00001F0180122FA01F0CB40C1F12001DBB2B9
:1015B000C0B2C01A2CFA01F3D11A914311EAC31137
:1015C000E6D1704701491820ABBEFEE726000200B5
:1015D00070475FEA400C08BF91F0000F4FEA8C2380
:1015E0004FEAC12243EA51514FEA1C5018BF00F59F
:1015F000F0404FEA300018BF41F000415FEA6C5CF8
:1016000000F02980BCF1FF3F08BF40F080407047E8
:10161000130C06BF12044FF0100C4FF0000C130E09
:1016200004BF12020CF1080C130F04BF12010CF1DD
:10163000040C930F04BF92000CF1020CD30F04BFF3
:1016400052000CF1010C11464FF00002A0F11F00F6
:10165000A0EB0C00704711F0004F08BF704731F04D
:1016600000413FF4D5AF0B0C06BF09044FF0100C3E
:101670004FF0000C0B0E04BF09020CF1080C0B0F0D
:1016800004BF09010CF1040C8B0F04BF89000CF19D
:10169000020CCB0F04BF49000CF1010CCCF120036C
:1016A000A0EB0C0022FA03F302FA0CF241EA030168
:1016B00000F10100704720F07F4C80EA030023F026
:1016C0007F47ACEB070303F57C5300F0004003F1C8
:1016D000FF032DE980494FEA154B09B44FEA144343
:1016E00025EA0B4E24EA03480FF2042606EB1327E3
:1016F00049083E785FEA320203FB0667C7F5000738
:1017000007FB06F64FEA54374FEAD64606F10206C3
:1017100007FB066CCCF1005C4FEA1C472CEA074C37
:1017200007FB06F40CFB06F504EB15464FEA96168C
:1017300034BF00204FF000404FEAD13706FB07FCD2
:101740004FEA1C4C0CFB0BF7D21B03FB0CF761EBB5
:1017500007010CFB0EF7B0EB074072EB17420CFBD6
:1017600008F734BFA2EB0742B2EB074261EB174127
:101770004FEA0C444FEA910706FB07FC4FEA1C4C6A
:101780000CFB0BF7B0EBC74072EB573203FB0CF7C7
:1017900034BFA2EBC742B2EBC74261EB57310CFB3F
:1017A0000EF7B0EBC70072EB57720CFB08F734BFB3
:1017B000A2EBC702B2EBC70261EB5771039F4FEA7E
:1017C000816141EA921104EBCC044FEAD1374FEA30
:1017D000826206FB07FC42EA90124FEA80604FEA01
:1017E0001C4C0CFB0BF7D21B03FB0CF761EB070146
:1017F0000CFB0EF7B0EB074072EB17420CFB08F73F
:1018000034BFA2EB0742B2EB074261EB17414FEA4C
:101810008C554FEA910704EB9C2406FB07FC4FEA2A
:101820001C4C0CFB0BF7B0EBC74072EB573203FBC1
:101830000CF734BFA2EBC742B2EBC74261EB5731A2
:101840000CFB0EF7B0EBC70072EB57720CFB08F7FE
:1018500034BFA2EBC702B2EBC70261EB577115EBC5
:101860004C254FEA816141EA92114FEA82624FEAC8
:10187000D13742EA901206FB07FC44F100044FEA1C
:1018800080604FEA1C4C0CFB0BF7D21B03FB0CF7E0
:1018900061EB07010CFB0EF7B0EB074072EB174250
:1018A0000CFB08F734BFA2EB0742B2EB074261EB37
:1018B000174115EB1C154FEA813141EA92414FEA7D
:1018C000823242EA90424FEA80304FEA0C7644F18D
:1018D000000448EA03434EEA0B484FF0000EB2EB17
:1018E000080C71EB030724BF624639464EEB0E0E1F
:1018F0004FF0000B0018524149414BEB0B0BB2EB80
:10190000080C71EB03077BF1000B24BF62463946DC
:101910004EEB0E0E4FF0000B0018524149414BEBBD
:101920000B0BB2EB080C71EB03077BF1000B24BF30
:10193000624639464EEB0E0E51EA020718BF46F0DA
:10194000010616EB0E7655F1000254F1000103D5A5
:10195000BDE88901BDE80088BDE88901BDE800480F
:10196000B619524141EB0101A3F101037047808098
:101970007F7E7D7C7B7A79787776767574737271E9
:1019800071706F6E6E6D6C6C6B6A6A6968686766A1
:1019900066656464636362616160605F5F5E5E5D33
:1019A0005D5C5C5B5B5A5A595958585757565655A7
:1019B00055555454535352525251515050504F4F09
:1019C0004F4E4E4D4D4D4C4C4C4B4B4B4A4A4A4959
:1019D000494948484847474747464646454545449C
:1019E0004444444343434342424242414141002B29
:1019F00026D4770021D01CB54FEA370703B44FF047
:101A000010004FF010014FF000000FBCBDE8104077
:101A10000BF1010BBBF1010F08BF5FEA170722BFF3
:101A200012F1010211F101014FF0004143F10003F5
:101A300000F0004043EA00007047F9D35708DAE7A6
:101A400046EA064613F1400F4FEA16461FDD13F132
:101A5000200FDFBF16430A46002120335B42C8D067
:101A6000C3F1200746EA064602FA07F74FEA164690
:101A700046EA0706C3F1200722FA03F201FA07F744
:101A800021FA03F14FF0000342EA0702B1E746EA08
:101A9000020646EA06464FEA164646EA0106BCBF7B
:101AA00046EA0646360C4FF000034FF000024FF0B6
:101AB00000019EE72DE9C048934630B491E8380014
:101AC00007C831EA400C48BF34EA430C03D5FFF79E
:101AD000F2FDFFF78CFFF0BCBDE800882DE9C0489F
:101AE000934630B491E8380007C810F0804F08BF23
:101AF00013F0804F03D100F005F8FFF778FFF0BC3A
:101B0000BDE8008820F07F4780EA030023F07F4C87
:101B100007EB0C03A3F57C5300F00040A3F1FE0398
:101B200092F0000F00F0B38095F0000F00F0778086
:101B30002DE901494FEA11404FEA144621EA0048D5
:101B400000FB06FC24EA064708FB06F607FB08F83C
:101B500000FB07F718EB06484CEB164C4FEA124B0C
:101B600018EB07484FEA15464CEB174022EA0B4E9C
:101B70000BFB06FC25EA06470EFB06F607FB0EFEEE
:101B80000BFB07F71EEB064E4CEB164C4FF0000616
:101B90001EEB074E4CEB174B18EB0B0840F1000007
:101BA00018EB0E0B58EB000840F100008F1A4FF0B5
:101BB00000013CBFC943661B14BFB5EB040C0021F8
:101BC0003CBFC943F61B4FEA17444EEA8E0E27EA84
:101BD00004454FEA1C4704FB07622CEA074C05FB4F
:101BE00007F70CFB05F604FB0CFC16EB074642EB73
:101BF000174216EB0C4642EB1C421BEB060658EB59
:101C00000202414146EA9E0601D5BDE80189B619A6
:101C1000524141EB0101A3F10103BDE801894FEA03
:101C200014454FEA114724EA054621EA074C05FB13
:101C300007F406FB07F70CFB06F105FB0CFC11EBA8
:101C4000074144EB17444FEA124711EB0C4144EBB8
:101C50001C4422EA074C05FB07F206FB07F70CFBC6
:101C600006F605FB0CFC16EB074642EB174216EB9B
:101C70000C4642EB1C456A1854F1000148BF7047FE
:101C8000B619524141EB0101A3F10103704795F0F0
:101C9000000F37D04FEA11424FEA144721EA0246BB
:101CA00024EA074C02FB07F106FB07F70CFB06F4DE
:101CB00002FB0CFC14EB074441EB17414FEA1547BC
:101CC00014EB0C4441EB1C4125EA074C02FB07F5E1
:101CD00006FB07F70CFB06F602FB0CFC16EB0746AF
:101CE00045EB174516EB0C4645EB1C42121951F11A
:101CF000000148BF7047B619524141EB0101A3F101
:101D0000010370474FEA14454FEA114724EA05469C
:101D100021EA074C05FB07F106FB07F70CFB06F26F
:101D20004FF0000605FB0CFC12EB074241EB17419C
:101D300012EB0C4251EB1C4148BF7047921841EB2B
:101D40000101A3F1010370472A4808B5816941F0F8
:101D500004018161816901F004010091816941F40C
:101D600000718161806900F4007000902248016870
:101D700021F00F0101602148016841F00701016075
:101D80001E480021243001601C480838026842F0D7
:101D9000010202604FF4FA530091009A521C009223
:101DA0009A42FAD3026842F00802026002681207FF
:101DB000FCD4026842F00402026002685207FCD4BC
:101DC000026842F4F0120260026842F4800202608B
:101DD0000A4800910A4910380268920704D4009A10
:101DE000521C00928A42F7D304483C30006880B20B
:101DF00008BD00000010024000080140102401400E
:101E0000A086010070B5FFF79FFF40F293440146A2
:101E1000A04214D20AA002F0E3FD4FF4FA75144870
:101E200000F049FE284600F0F7FCFFF78DFF014661
:101E3000A042F4D3BDE870400EA002F0C1BD70BD59
:101E40005B424C5D20D6F7B5E7D4B4CEB4C9CFB56C
:101E5000E720284144433D257529A3ACB5C8B4FD0E
:101E60002031325620BBD6B8B42E2E2E00000000F2
:101E7000980400205B424C5D20D6F7B5E7D4B4D27D
:101E8000D1BBD6B8B420284144433D257529000074
:101E9000FEE700002DE9F0470F460A46814601465D
:101EA00000252BA002F08CFD4FF4806644E0781BE7
:101EB0003446A04200D80446314800F0FCFD4FF4FF
:101EC0000051304800F0BBFD2F4830492B18C4F3B7
:101ED0008F02002005E000BF53F820C041F820C069
:101EE000401C9042F8DBDFF8A4C000200CF58063B2
:101EF00011E000BF5CF8201003EB800203F8201013
:101F00004FEA112882F801804FEA1148090E82F841
:101F10000280D170401CB0EB940FEBD309EB0500AD
:101F2000804622461A4902F028FC404622461849BB
:101F300002F0DEFB28B12544BD42B8D30120BDE844
:101F4000F08709EB050113A002F02AFD0020F6E757
:101F50005B424C5D20B1B8B7DD2041505031202D9F
:101F60003E20CDE2B2BF20466C61736820307825F8
:101F7000303658A3ACB4F3D0A13D25750000000065
:101F8000980400200010014000800008E80C0020A8
:101F9000E81000205B4641494C5D205732355136F0
:101FA0003420B1B8B7DDD0A3D1E9CAA7B0DC204056
:101FB00030782530365800002DE9F0470F460B46A3
:101FC000314E824601460024324630A002F0F8FC31
:101FD0004FF48069DFF8E8804EE03D1B4D4500D9A5
:101FE0004D46384800F067FD4FF40051364800F088
:101FF00026FD0AEB04002A46344902F0C5FA002007
:10200000324A08E002EB8001CB78096863F31F6174
:1020100048F82010401CB0EB950FF3D3AA082849CC
:10202000A01902F0DDFB10B10020414615E0A11916
:1020300027A002F0B5FC0CE004EB8002935951F8A4
:1020400020209A4208D004EB8000811927A002F0DA
:10205000A7FC0020BDE8F087401CB0EB950FEBD348
:102060002C44A00408D164206043B0FBF7F3BA0A03
:10207000A10A2CA002F0A4FCBC42AED32FA002F017
:102080009FFC0120E6E70000008000085B424C5DF9
:1020900020BFBDB1B4CDE2B2BF20466C61736820F1
:1020A000307825303658202D3E2041505031203098
:1020B0007825303858A3ACB4F3D0A13D2575000085
:1020C000E80400209804002000100140E8080020E7
:1020D0005B4641494C5D20D0B4C8EB2041505031A3
:1020E00020CAA7B0DC204030782558005B46414923
:1020F0004C5D20D0A3D1E9204150503120CAA7B077
:10210000DC204030782558A3BA77726F74653D3073
:10211000782530385820726561643D307825303834
:10212000580000003E20BDF8B6C83A2025752F257E
:1021300075204B4220282575252529005B204F4B13
:10214000205D20BFBDB1B4CDEAB3C900014800F0A5
:10215000C9B90000A404002030B590F84050012413
:10216000AC40C56B6C60046863604368102B036807
:1021700003D099600068C26030BD9A600068C16099
:1021800030BD70472DE9F047824602460E4629A031
:1021900002F016FC002534274FF4FA792D4C41E06B
:1021A0000AEBC5282C4800F086FC4FF400512B4860
:1021B00000F045FC00F086F8E760484600F092F831
:1021C000F8B1206940F002002061C4F81480206951
:1021D00040F040002061484600F084F8B0B1E26869
:1021E000206920F002002061D00618D541461CA0CD
:1021F00002F0D6FBC4F80C7000F05CF80020BDE8DB
:10220000F08741461DA002F0CBFBF5E741461BA03D
:1022100002F0C6FB206920F002002061ECE700F02C
:1022200049F86D1CB542BBD331461CA002F0C8FB77
:102230000120E4E73E20B2C1B3FD20257520D2B3D2
:10224000A3ACC6F0CABCB5D8D6B720307825582E76
:102250002E2E0000002002409804002000100140B3
:102260003E20B2C1B3FDCAA7B0DC2040307825586B
:10227000A3BA53523D307825580000003E20B2C129
:10228000B3FDCAA7B0DC204030782558A3BAC3A656
:10229000B5C8B4FDB3ACCAB1000000003E20B2C165
:1022A000B3FDCDEAB3C9A3A8257520D2B3A3A90075
:1022B00072B6FEE70248016941F080010161704792
:1022C0000020024004480169090603D50349416022
:1022D0000349416070470000002002402301674528
:1022E000AB89EFCD70B5054600F0B6FB0446074E4E
:1022F00007E000BF00F0B0FB001BA84201D900209E
:1023000070BDF068C007F5D1012070BD002002400B
:102310002DE9F0410E460746FFF7D4FF124C342555
:10232000E5606420FFF7DEFF80B1206940F0010026
:1023300020613E806420FFF7D5FF60B1E06821692D
:1023400021F001012161E560C00609D5FFF7B2FF68
:102350000020BDE8F081206920F001002061F5E750
:10236000FFF7A8FF0120F4E70020024010B590F825
:1023700021100022022905D00421816380F8202049
:10238000012010BD01680B6823F00E030B6001688B
:102390000B6823F001030B6090F84030C46B0121FF
:1023A00001FA03F3636080F8211080F820201046C2
:1023B00010BD00002DE9F05F90F8211000240229E3
:1023C00003D004218163012485E001680A6822F0BA
:1023D0000E020A6001680A6822F001020A603F4E9C
:1023E0003E4FB215DFF8F4C0DFF8F090DFF8ECA054
:1023F000DFF8E8B0DFF8E4E00168783F1301150288
:10240000ACF1640CA9F15009AAF13C0AABF1280B1C
:10241000AEF1140E4FF48018B14227D9B9420ED054
:10242000614512D049451DD0514518D0594518D0A5
:10243000714501D1424615E0294EB14201D1012238
:1024400010E0274E1436B14201D110220AE0244E8A
:102450002836B14206D0224A3C32914201D11A4676
:1024600000E02A461E49091F0A602BE0B94213D03A
:10247000614517D0494522D051451DD059451DD041
:10248000714501D142461AE0B14202D14FF080724B
:1024900015E0134EB14201D1012210E0104E143666
:1024A000B14201D110220AE00D4E2836B14206D0C9
:1024B0000B4A3C32914201D11A4600E02A460749B4
:1024C00080394A60012180F82110002180F8201015
:1024D000416B01B188472046BDE8F09F8000024073
:1024E000080402402DE9F05FC16B0A6801680B68BF
:1024F000046C4FF0040808FA04F8844D844E854FAC
:10250000DFF814C2DFF81492DFF814A2DFF814B277
:10251000DFF814E218EA020F65D05FEA437862D56B
:102520000A68920603D40A6822F004020A60DFF8FF
:10253000F0814FF48062016808F11408130114025D
:10254000414524D9A9420DD0B1420FD0B9421AD089
:10255000614515D0494515D0514501D1120312E00E
:10256000594501D104220EE0714501D140220AE013
:102570006D4D1435A94206D06B4A2832914201D1E3
:102580001A4600E022466749091F0A6029E0A9426D
:1025900013D0B14215D0B94220D061451BD0494576
:1025A0001BD0514502D14FF4800217E0414502D1C2
:1025B0004FF0806212E0594501D104220EE07145CE
:1025C00001D140220AE0584D1435A94206D0564A9E
:1025D0002832914201D11A4600E022464B4908397F
:1025E0004A60C16A71E04FF0020808FA04F818EA7C
:1025F000020F70D05FEA83786DD50A68920606D420
:102600000A6822F00A020A60012180F82110DFF82E
:1026100010814FF40072016808F1140813011402CC
:10262000414524D9A9420DD0B1420FD0B9421AD0A8
:10263000614515D0494515D0514501D1120312E02D
:10264000594501D102220EE0714501D120220AE054
:10265000354D1435A94206D0334A2832914201D172
:102660001A4600E022462F49091F0A6029E0A942C4
:1026700013D0B14215D0B94220D061451BD0494595
:102680001BD0514502D14FF4001217E0414502D151
:102690004FF0007212E0594501D102220EE071455F
:1026A00001D120220AE0204D1435A94206D01E4A4D
:1026B0002832914201D11A4600E0224613490839D6
:1026C0004A60002180F82010816A00291CD0BDE8F2
:1026D000F05F0847FFE70825A540154214D01A0708
:1026E00012D50A6822F00E020A6090F84020C36BEF
:1026F000012101FA02F25A60816380F82110002161
:1027000080F82010016BE0E7BDE8F09F0800024070
:102710001C000240300002404400024058000240C9
:102720006C000240080402401C04024030B560B155
:102730001A4B026814219A4209D2194B1344B3FB75
:10274000F1F18900016417490AE0012030BD134B03
:102750005B421344B3FBF1F1890001640F4908396E
:10276000C163022180F82110136843F6F0718B4396
:10277000F0E901142143D0E902452C4321430469C7
:102780002143446921438469214319431160002195
:102790004163012242770177084630BD08040240B8
:1027A000F8FFFDBF0000024070B5044690F820001D
:1027B000002501280CD0012084F8200094F8216025
:1027C0000020012E06D084F820000225284670BD86
:1027D000022070BD022684F82160A063206806688C
:1027E00026F0010606602046FFF7B6FCE06A0028E6
:1027F0002068016802D041F00E0106E021F00401DA
:1028000001602068016841F00A01016020680168E8
:1028100041F001010160D9E770B5044600F01CF9F0
:102820000546601C02D004480078044400F014F906
:10283000401BA042FAD370BD040000202DE9F84FE0
:10284000DFF8C891002409F1040A0AF1040B2346B9
:102850000F270BF1040ED1E00125A54006EA050281
:10286000AA4276D1DFF8A8C14E68A6EB0C086645EF
:102870002BD00DDC032E34D005DC36B3012E19D05D
:10288000022E2FD11BE0112E16D0122E2AD119E0C4
:10289000B8F5881F19D006DCB8F5803F15D0B8F51B
:1028A000801F1FD111E0B8F5001F0ED0B8F5041F2E
:1028B00018D10AE0CB6815E0CB681B1D12E0CB688D
:1028C00008330FE0CB680C330CE08B682BB1012B85
:1028D0004FF0080303D0456104E0042302E00561E2
:1028E00000E00023FF2A01D8064601E000F10406BB
:1028F0004FEA840501D9A5F12005D6F8008007FA32
:1029000005FC28EA0C0803FA05F548EA0508C6F8AC
:1029100000804D68ED0070D53E4DAE6946F0010671
:10292000AE61AD6924F0030605F0010500953A4D4E
:1029300006EB050CDCF80850A607360F07FA06F878
:1029400025EA0805DFF8D480404503D14FF00008A0
:1029500025E052E0DFF8C880404502D14FF0010881
:102960001DE0DFF8C080404502D14FF0020816E0BC
:10297000DFF8B480404502D14FF003080FE0DFF8E4
:10298000AC80404502D14FF0040808E0DFF8A08099
:10299000404502D14FF0050801E04FF0060808FA63
:1029A00006F848EA0508CCF808804D68D9F80060B8
:1029B000ED034D4601D5164300E096432E604D6869
:1029C000DAF80060AD03554601D5164300E09643A2
:1029D0002E604D68DBF80060ED025D4601D51643C0
:1029E00000E096432E604D68DEF80060AD0275464B
:1029F00001D5164300E096432E60641C0A68164613
:102A0000E2407FF429AFBDE8F88F000000040140E8
:102A100000001110001002400000014000080140B9
:102A2000000C01400010014000140140001801405A
:102A3000001C01408068084000D001207047C26837
:102A40000A4201D041617047016170470AB10161DA
:102A500070470904FBE700000148806870470000E8
:102A60000400002070B5040011D021684CF6CC4061
:102A70000860216845F255500860D4E900014160C2
:102A80002168A0688860FFF7E7FF054609E001209C
:102A900070BD00BFFFF7E0FF401B302801D90320C5
:102AA00070BD2068C0680028F4D121684AF6AA20C9
:102AB0000860002070BD00684AF6AA21016000206D
:102AC00070470000024881680278114481607047B5
:102AD00004000020074810B5016841F010010160B2
:102AE000032000F085F8002000F006F800F024F83C
:102AF000002010BD0020024070B50D4D04464FF47B
:102B00007A712878B1FBF0F00A490968B1FBF0F05E
:102B100000F0FCFA48B9102C07D200222146501EC2
:102B200000F046F800206C6070BD012070BD000010
:102B300004000020100000200C4808B5816941F015
:102B400001018161816901F001010091C16941F0D8
:102B50008051C161C06900F0805000900448416814
:102B600021F0E06141F00071416008BD00100240B9
:102B70000000014000280DDB00F01F020121914000
:102B80004009800000F1E020C0F88011BFF34F8FB2
:102B9000BFF36F8F7047002809DB00F01F0201218F
:102BA00091404009800000F1E020C0F8001170471A
:102BB000F0B40E4B1B680C46C3F30223C3F10705A8
:102BC000042D00D90425191D072901D2002300E096
:102BD000DB1E012606FA05F1491E214099409E4060
:102BE000761E16403143F0BC01F069BE0CED00E0EA
:102BF000064900F0070208684FF6FF03184040EA54
:102C00000220034A10430860704700000CED00E00A
:102C10000000FA052DE9F0470F46050061D0434E4C
:102C2000306800F00700B84209D2306820F0070091
:102C300038433060306800F00700B84251D128684E
:102C40003B4C810712D5400703D5606840F4E06033
:102C500060602878000703D5606840F460506060C9
:102C60006068A96820F0F000084360602878C00719
:102C700028D06868012810D02168022810D0890760
:102C800000292EDA616821F0030101436160FFF73A
:102C9000E3FE804641F288390DE021688903EFE7C1
:102CA0008901EDE7FFF7D8FEA0EB0801494502D9FD
:102CB0000320BDE8F0876068696800F00C00B0EBA5
:102CC000810FEFD1306800F00700B8420BD93068AF
:102CD00020F0070038433060306800F00700B84249
:102CE00001D00120E5E72878400705D56068E9684C
:102CF00020F4E060084360602878000706D560682B
:102D0000296920F4605040EAC100606000F038F8A2
:102D10006168084AC1F30311515CC8400649086064
:102D200006480068FFF7E8FE0020C2E700200240E6
:102D300000100240584B000810000020080000203E
:102D40000448054900684968044AC1F30221515CFE
:102D5000C84070471000002000100240684B000877
:102D60000448054900684968044AC1F3C221515C1E
:102D7000C84070471000002000100240684B000857
:102D800012A185B00FC98DE80F0014A0144A006885
:102D900004905168134801F00C03042B10D0082B49
:102DA0000ED1C1F38343C9031DF803000AD551684E
:102DB00004AAC1F34041515C0A4A5043B0FBF1F010
:102DC00005B0704708494843FAE7000002030405CC
:102DD000060708090A0B0C0D0E0F10100102000067
:102DE0000010024000127A0000093D002DE9F84F62
:102DF000040070D02078C04DC00749D06868C0F387
:102E00008100012807D06868C0F38100022809D139
:102E10006868C00306D52868800339D56068002833
:102E2000E7D035E06068B0F5803F0BD010B1B0F569
:102E3000A02F11D0286820F480302860286820F462
:102E4000802002E0286840F480302860606890B1FB
:102E5000FFF702FE06460AE0286840F4802028605A
:102E6000F0E700BFFFF7F8FD801B642873D82868DF
:102E70008003F7D50CE0FFF7EFFD064605E000BF45
:102E8000FFF7EAFD801B6428F0D828688003F7D498
:102E900020789A4E80074FF001094FF0000839D58D
:102EA000686810F00C0F07D06868C0F38100022832
:102EB00009D16868C00306D42868800714D5206942
:102EC000012808D110E02069B0B1C6F80090FFF7E2
:102ED000C3FD074605E00AE1FFF7BEFDC01B02285F
:102EE000C4D828688007F7D52868616920F0F80001
:102EF00040EAC10028600DE0C6F80080FFF7ACFD95
:102F0000074604E0FFF7A8FDC01B022823D8286865
:102F10008007F7D4207800072CD57948A169D9B16A
:102F2000C0F80090FFF798FD074604E0FFF794FD16
:102F3000C01B02280FD8686A8007F7D571484FF484
:102F4000FA510068B0FBF1F0009000BF0098411EFC
:102F50000091FAD20EE080E0C0F80080FFF77CFD1F
:102F6000074604E0FFF778FDC01B022875D8686AA1
:102F70008007F7D42078400760D5E8690027C000B3
:102F800008D4E86940F08050E861E869012700F062
:102F9000805000905C480168C90513D401688346DD
:102FA00041F480710160FFF757FD824606E000BFE3
:102FB000FFF752FDA0EB0A0064284ED8DBF80000B2
:102FC000C005F5D5E06801280AD008B1052813D05E
:102FD000286A20F001002862286A20F0040002E03C
:102FE000286A40F001002862E06841F2883B98B10D
:102FF000FFF732FD82460BE0286A40F004002862A9
:10300000EEE700BFFFF728FDA0EB0A0159455AD8AB
:10301000286A8007F6D50CE0FFF71EFD824605E022
:10302000FFF71AFDA0EB0A0159454CD8286A800722
:10303000F6D41FB1E86920F08050E861E06988B3F8
:103040006968C1F38101022944D00228C6F8608072
:1030500004D0FFF701FD044638E034E0FFF7FCFC44
:10306000074604E0FFF7F8FCC01B02282BD82868AD
:103070008001F7D4206AB0F5803F05D16868A16867
:1030800020F4003008436860D4E908010843696807
:1030900021F4741108436860C6F86090FFF7DCFC07
:1030A000044606E025E000BFFFF7D6FC001B02281F
:1030B00009D828688001F7D51BE000BFFFF7CCFCDA
:1030C000001B022802D90320BDE8F88F2868800180
:1030D000F4D40EE00128F7D06868226A00F4803149
:1030E000914204D1616A00F47010884201D001203D
:1030F000EAE70020E8E7000000100240000042423A
:1031000080044242100000200070004010B5401EB4
:10311000B0F1807F01D3012010BD4FF0E024606149
:103120000F21601701F0CBFB0020A0610720206178
:10313000002010BD10B504460068416994F839209C
:10314000C1F3C011212A0BD151B1416921F0800195
:103150004161206B08B1FFF709F9204600F0B6FE87
:103160002068416994F83A20C1F38011222A0BD1DA
:1031700051B1416921F040014161606B08B1FFF735
:10318000F5F8204600F094FE002010BD70470000C6
:1031900070B5026804461068D168536910F00F0FCB
:1031A00051D003F0010501F4907635435DD0C2079C
:1031B00005D0CA0503D5E26B42F00102E263420783
:1031C00005D5DA0703D0E26B42F00202E263820720
:1031D00005D5DA0703D0E26B42F00402E26302078E
:1031E00005D5DA0703D0E26B42F00802E263E26B36
:1031F000002A34D0800604D5880602D5204600F087
:103200006EFE20684069E16BC0F3801001F0080198
:103210000143204624D000F04BFE20684169490656
:103220001AD5416921F040014161606BA0B11B4991
:103230004163606BFFF7BEF8002810D0606B416BF4
:10324000BDE87040084783060FD58B060DD5204694
:10325000BDE8704000F043BE2046FFF797FF70BD09
:10326000FFF794FF0020E06370BD030606D50B0650
:1032700004D52046BDE8704000F0D8BE4006F3D526
:103280004806F1D5D168204621F04001D1602021C7
:1032900084F8391000F061F970BD0000113E00089B
:1032A00070B5040004D094F83900002510B106E090
:1032B000012070BD84F83850204600F023F8242007
:1032C00084F839002068C16821F40051C1602046AB
:1032D00000F050FE2068016921F4904101612068EE
:1032E000416921F02A0141612068C16841F400511F
:1032F000C160E563202084F8390084F83A0000209A
:1033000070BD0000F0B585B00024009401940294D3
:10331000039406460368344F0220344903224502D1
:10332000BB4221D18B6943F480438B618B6903F4E9
:10333000804304938B6943F004038B6189692C4EAD
:1033400001F0040104910102CDE9001003926946E5
:103350003046FFF773FACDE90054694630460294CF
:10336000FFF76CFA05B0F0BD224FBB42FAD1CB6932
:1033700043F48023CB61CB6903F4802304938B69EE
:1033800043F008038B61896901F00801CDE903214D
:10339000CDE90050184D69462846FFF74FFAE8146A
:1033A000CDE90004694628460294FFF747FA144D18
:1033B0001248C5E900048020C5E902402C616C6117
:1033C000AC612846EC61FFF7B1F908B1FEF770FF78
:1033D00075630022012127206E62FFF7E9FB272099
:1033E000FFF7D9FBBEE700000038014000100240A3
:1033F0000008014000480040000C0140300002403D
:10340000A4040020F8B5044690F83A0020283CD1E6
:10341000C1B3BAB394F83800012836D0012084F83B
:103420003800A162A2850025E563222084F83A00D5
:10343000636B17489862636B1648D862636B1648D3
:103440001863606B134645630846666B2168024645
:103450003046091DFFF7A8F920680168416800910E
:1034600084F83850C16841F48071C16020684169B6
:1034700041F0010141612068416941F04001416131
:103480000020F8BDFFE70120FBE70220F9E700007C
:103490006B3E0008A73E0008213E000870477047B9
:1034A0002DE9F843044690F839001F4616460D46AC
:1034B000202850D1A5B19EB194F8380001284AD0F7
:1034C000012084F838004FF00008C4F83C80212027
:1034D00084F83900FFF7C0FAA6848146E68426E026
:1034E0000120BDE8F883E08C401EE084A0684B46D4
:1034F000B0F5805F4FF000024FF08001204600974A
:1035000003D000F0C4FDE8B90DE000F0C0FDC8B97B
:1035100028882168C0F308004860206908B16D1C44
:1035200005E0AD1C03E0216815F8010B4860E08C54
:103530000028D8D14B46002240212046009700F0B9
:10354000A6FD08B10320CCE7202084F8390084F8D8
:1035500038800020C5E70220C3E77047FEE700007F
:1035600070B501681A4A1140B1F1005F05D0BDE89D
:103570007040014617A001F013BA0568446801467F
:103580001EA001F01DFA2548FFF7D4FD234800686E
:10359000C16821F01001C1602720FFF7EBFA0D2070
:1035A000FFF7E8FA272001F07DF90D2001F07AF904
:1035B0004FF0E0210020086119494FF000700860C9
:1035C0002846FCF759FEA446BDE87040604700005D
:1035D0000000FE2F5B424C5D20B4EDCEF3A3BA4158
:1035E0005050204030782530385820D5BBB6A5B58E
:1035F000D8D6B7B7C7B7A8A3A10000005B424C5DFF
:1036000020D5FDD4DACCF8D7AAB5BD204150503131
:1036100020403078253038582E2E2E0058040020B7
:1036200004ED00E000B585B0002002901D488169DE
:1036300041F020018161816901F0200104918169DB
:1036400041F004018161816901F004010491816903
:1036500041F008018161816901F0080104918169EB
:1036600041F010018161816901F0100104918169CB
:1036700041F001018161806900F0010004900A4875
:10368000416821F0E06141F0007141604014009018
:10369000012001900220039069460448FFF7CEF80C
:1036A00005B000BD001002400000014000100140C4
:1036B000FEE77047704770472DE9F0478CB0BFA018
:1036C00001F07EF9BEA001F07BF9C6A001F078F907
:1036D000CD480188CDA001F073F9D5A001F070F9B3
:1036E0004FF40051DB48FFF7AAF9DB48446A416A0E
:1036F00041F080714162D94D2868D94EDFF85C9362
:10370000002705F1040809F110094FF0010AB04241
:1037100009D1284601F024F9D9F80010884202D1D5
:10372000C8F8004007E0CD4808300760001D07607A
:10373000C8F800402E60284601F012F9C9F80000D0
:10374000600001D5C7A000E09CA0A10001D5C8A1E0
:1037500000E09AA1CDE90010E00001D5C7A300E088
:1037600096A3600101D5C7A200E094A2200101D573
:10377000C6A100E091A1C7A001F022F9FEF742FB2B
:1037800002A800F04DFECB4D4FF4603600287DD1ED
:103790009DF81800002819D09DF81900012801D0C3
:1037A000022814D1DDF8121039B1DDF81210B1423F
:1037B00003D89DF81210890709D0DDF81210BEA0B9
:1037C00001F00EF900F0FCFD8DF818707BE0012887
:1037D00001D0022877D1BDF81630DDF81220BDF8EF
:1037E0001010C0A001F0ECF8022000F063FE31469A
:1037F000284600F0ABFC07469DF8260008B12FB321
:103800002CE01FB3C5A001F0DBF83146002000F02A
:103810000CFD3146284601F0ABF8804631460020C9
:10382000FEF738FB20B14146304600F02AFE30B1A9
:10383000BFA001F0B5F8012000F03CFE09E08DF8D2
:1038400026A04146C8A001F0BBF802E0CDA001F0DF
:10385000C7F89DF8260008B9002F34D1D6A001F092
:10386000AFF870212846FEF78DFC30B3DDF812105A
:103870004FF48020FEF7A0FBF8B1DDF812102846C7
:1038800001F076F80746BDF8161000E077E0B9427F
:103890000FD1DDF81210284600F058FC48B1394627
:1038A000CBA001F08DF8032000F004FE00F074FDC1
:1038B0006AE03946D1A001F073F8DCA001F090F87D
:1038C000012000F0F7FD9DF81900032849D19DF86B
:1038D0001C0028B1E0A001F073F800F071FD40E099
:1038E00014F0C04F0BD000F085FDBDF81A00401C4D
:1038F00081B2ADF81A10E0A001F072F803E02146A1
:10390000E8A001F05DF8BDF81A00032829D3F0A063
:1039100001F066F89DF8260000B30898F0B1B042B7
:103920001CD880071AD170212846FEF72BFCA8B1BD
:1039300000200899FEF740FB80B12846089901F065
:1039400017F8BDF82410814208D13146284600F00E
:10395000FDFB18B1042000F0ADFD15E0E6A001F07C
:103960001FF89DF81900042809D13146284600F0B7
:10397000EDFB48B9E4A001F033F800F021FD314639
:10398000284600F0E3FB28B12846FFF7E9FD0CB01C
:10399000BDE8F087E7A001F003F840F6B830FEF785
:1039A0003BFFBFF34F8FED480168ED4A01F4E06142
:1039B00011430160BFF34F8F00BFFDE7000000001F
:1039C0002A202A202A202A202A202A202A202A20A7
:1039D0002A202A202A202A202A202A202A202A2097
:1039E0002A202A002A2020202020202020202020D9
:1039F000426F6F744C6F616465722020202020201C
:103A00002020202020202A00E0F7FF1F2A2020204D
:103A10002020202020202020466C6173683A202539
:103A2000644B4220202020202020202020202A001B
:103A30002A202A202A202A202A20202020427920D9
:103A400048656C65692020202A202A202A202A2007
:103A50002A202A00001001400010024000BF002070
:103A6000524853522057574447BFB4C3C5B9B70053
:103A70002049574447BFB4C3C5B9B70020C8EDBCFF
:103A8000FE00000020B0B4BCFC00000020C9CFB58F
:103A9000E70000005B424C5D20C9CFB4CEB8B4CE85
:103AA000BBD4ADD2F23A25732573257325732573E4
:103AB00000000000008000085B424C5D20D0C2B9CD
:103AC000CCBCFEB4F3D0A1B7C7B7A8206E65775FB2
:103AD00073697A653D2575A3ACB6AAC6FAD0C2B99A
:103AE000CCBCFE005B424C5D20CDE2B2BF20466CF8
:103AF00061736820D6D0D3D0D0C2B9CCBCFEA3BAF3
:103B00007665723D25752073697A653D257520635C
:103B100072633D3078253034580000005B424C5DC4
:103B200020B2C1B3FDB1B8B7DDB2DB2E2E2E00003E
:103B30005B424C5D20B1B8B7DDCAA7B0DCA3ACB71F
:103B4000C5C6FAB8FCD0C2A3A8B1A3C1F4BEC920AF
:103B500041505031A3ACCFC2B4CEC6F4B6AFD6D824
:103B6000CAD4A3A9000000005B424C5D20B1B8B7E5
:103B7000DDCDEAB3C9A3AC6372633D307825303440
:103B8000580000005B424C5D204150503120CEDE99
:103B9000D0A7A3ACCEDEBFC9B1B8B7DDC4DAC8DDEB
:103BA000A3BBB8FCD0C2CAC7CEA8D2BBD7D4BEC8AC
:103BB000CAD6B6CE000000005B424C5D20D5FDD4D5
:103BC000DAB8FCD0C220415050312E2E2E00000019
:103BD0005B424C5D204150503120B8FCD0C2B3C98B
:103BE000B9A6A3AC6372633D307825303458A3ACDA
:103BF000CCF8D7AAD4CBD0D0000000005B424C5DFB
:103C000020415050312043524320BBF2CDB7B2BFC8
:103C1000D0A3D1E9B2BBC6A5C5E4A3A16170705F12
:103C20006372633D30782530345800005B424C5D50
:103C3000204150503120B8FCD0C2CAA7B0DCA3ACA0
:103C4000B1A3C1F4CDE2B2BFD0C2B9CCBCFED2D4D4
:103C5000B1E3D6D8CAD400005B424C5D20B8FCD09A
:103C6000C2D2D1C8B7C8CFA3ACC7E5C0ED204F546E
:103C70004120B1EAD6BE00005B424C5D204150506D
:103C800020BFA8CBC0A3A8BFB4C3C5B9B7B8B4CE32
:103C9000BBA3A9A3ACCAD4B4EDB4CECAFD3D25756F
:103CA000000000005B424C5D20CAD4D4CBD0D0C60B
:103CB000F4B6AFA3ACB8B4CEBBB1EAD6BE3D307853
:103CC00025303858A3A8B2BBBCC6CAFDA3A90000C2
:103CD0005B424C5D20B4EFB5BDD7EEB4F3CAD4B4AB
:103CE000EDB4CECAFDA3ACBBD8CDCBB5BDB1B8B792
:103CF000DDB9CCBCFE0000005B424C5D20BBD8CDE2
:103D0000CBCAA7B0DCA3A1005B424C5D20BBD8CDE1
:103D1000CBD7B4CCACB5AB204150503120CEDED0A7
:103D2000A7A3ACC7E5B3FD204F544120B1EAD6BEEE
:103D3000000000005B424C5D20CEB4D5D2B5BDD3AF
:103D4000D0D0A7B5C42041505031A3A1337320BABD
:103D5000F3B8B4CEBBD6D8CAD40000000CED00E056
:103D60000400FA05FEF7AEBE30B58FB028216846D4
:103D7000FCF772FB14210AA8FCF76EFB0121080472
:103D8000CDE900100024029402250491CDE90750EA
:103D90004FF4E01009906846FFF728F808B172B6B2
:103DA000FEE70F20CDE90A054FF48060CDE90C4015
:103DB00002210AA80E94FEF72DFF002801D072B64A
:103DC000FEE70FB030BD00000D48016841F0010171
:103DD000016041680B4A1140416001680A4A114084
:103DE0000160016821F480210160416821F4FE0135
:103DF00041604FF41F0181600449C00308607047AF
:103E0000001002400000FFF8FFFFF6FE08ED00E0A2
:103E100010B5406A0021C185C184FFF7B7F910BD14
:103E200070B5446A2068406994F83910C0F3C01036
:103E30000025212904D118B1E584204600F046F878
:103E40002068406994F83A10C0F38010222904D108
:103E500018B1E585204600F02BF8E06B40F010002B
:103E6000E0632046FFF792F970BD10B50146406A45
:103E700009680968890613D40021C1850168CA68E8
:103E800022F48072CA6001684A6922F001024A6124
:103E900001684A6922F040024A61202180F83A1004
:103EA000FFF7FCFA10BD10B5406AFFF7F8FA10BD35
:103EB0000168CA6822F49072CA6001684A6922F0F7
:103EC00001024A61202180F83A1070470168CA68EF
:103ED00022F0C002CA60202180F83910704710B566
:103EE00090F83A10222901D0022010BD8168B1F566
:103EF000805F11D00169002901681FD0496801F075
:103F00007F03816A4A1C82620B70C18D491E0904BD
:103F1000090CC18518D02BE00269816A002A026869
:103F2000526805D0D2B20A80816A491C8162ECE7EE
:103F3000C2F308020A80816A891CF7E74A68816A2D
:103F40004B1C83620A70E0E70168CA6822F0200215
:103F5000CA600168CA6822F48072CA6001684A694E
:103F600022F001024A61202180F83A10FFF796FA08
:103F7000002010BD2DE9F041044600680169E268A7
:103F800021F44051114301612169A068084361692E
:103F900008432168CA6841F20C639A430243CA602D
:103FA00020684169A26921F44071114341611E49B1
:103FB000206864253226884202D1FEF7D1FE01E056
:103FC000FEF7BEFE00EBC00101EB001160686FF070
:103FD00018078000B1FBF0F2B2FBF5F2B1FBF0F391
:103FE0007A4303EB8202B1FBF0F306EB0212B2FB61
:103FF000F5F2B3FBF5F302F0F00202EB0312B1FBB2
:10400000F0F3B1FBF0F0B0FBF5F0784303EB800088
:1040100006EB0010B0FBF5F0216800F00F00104433
:104020008860BDE8F08100000038014090F8391048
:10403000212901D0022070478168B1F5805F016AB3
:104040000BD04A1C0262026809785160C18C491E7B
:104050000904090CC1840ED017E009880268C1F375
:104060000801516001690029016A02D0491C0162FE
:10407000ECE7891CFBE70168CA6822F08002CA608D
:104080000068C16841F04001C160002070472DE91F
:10409000F041984617460E460446069D1DE0681CF2
:1040A0001BD02DB1FEF7D8FCA0EB0800A84214D914
:1040B0002068C16821F4D071C1602068416921F095
:1040C00001014161202084F8390084F83A00002081
:1040D00084F838000320BDE8F0812068006836EAE3
:1040E000000004D00020B842D9D00020F3E701201E
:1040F000F9E7000038B5104C20680168C943C906CB
:1041000014D40168406800902046FFF713F8606BF4
:10411000006840680949C0F58060088008490120AE
:104120008202087007492046FFF76CF9BDE8384065
:104130000148FFF72DB800005804002002000020BD
:104140000000002018000020FEE7000010B50A461D
:1041500001680C4B0B40B3F1005F01D00AA007E0EF
:1041600041681248814202D31044814204D910A010
:1041700000F016FC002010BD15A000F021FC01206D
:1041800010BD00000000FE2F3E20D0A3D1E9CAA739
:10419000B0DCA3BAD5BBB6A5B5D8D6B7B7C7B7A854
:1041A0002053503D30782558000000000080000862
:1041B0003E20D0A3D1E9CAA7B0DCA3BAB8B4CEBB25
:1041C000CFF2C1BFB7C7B7A83D307825580000006F
:1041D0003E20B9CCBCFED0A3D1E9CDA8B9FD0000EA
:1041E00070B5054600F0E2FA002816D10B4C00220B
:1041F00010212046FEF72AFCD82000F021FA28469C
:1042000000F0ACFA012210212046FEF71FFCBDE8A9
:10421000704041F2883000F08FBA70BD000C014050
:1042200000BF00BF00BF00BF704770B500291FD09E
:10423000451804466D1E04E0204600F039FA04F5E6
:1042400080542004000C01D0AC42F5D94FF6FF7623
:10425000A019A8420AD82046FFF7C2FF04F580340F
:10426000F6E7204600F024FA04F58054AC42F8D971
:1042700070BD024600200146535C491C184480B2C0
:104280002029F9D37047000010B50446006806499C
:10429000884207D12046FFF7ECFF218C884201D1EC
:1042A000012010BD002010BD4F5441572DE9F041B1
:1042B00086B0344800240294816941F00401816190
:1042C000816901F004010591816941F00801816172
:1042D000816901F008010591816941F00101816165
:1042E000806900F0010005902748416821F0E061F5
:1042F00041F0007141600320039001251020CDE9B9
:104300000005DFF8888069464046FEF797FA0820E6
:10431000009069464046FEF791FA1D4FEE0369464C
:1043200038460096FEF78AFA20208DE8310069466B
:104330004046FEF783FA012210214046FEF786FB35
:10434000002208214046FEF781FB00223146384614
:10435000FEF77CFB04A8049400F03AF99DF81000E5
:104360009DF81110000440EA01209DF81210084346
:104370000849884203D0012006B0BDE8F081002042
:10438000FAE700000010024000000140000C01406C
:10439000000801401740EF0000B589B0684600F002
:1043A0003FF818B14FF0FF3009B000BD0198401C34
:1043B000019000208DF81400684600F08FF8F3E7B4
:1043C00000B589B0684600F02BF818B14FF0FF3007
:1043D00009B000BD0198401C019000208DF810002C
:1043E0008DF811008DF814008DF81E00684600F05D
:1043F00075F8EDE700B589B0684600F011F818B11E
:104400004FF0FF3009B000BD0198401C0190BDF88D
:104410001200401CADF81200684600F05FF8F1E7AA
:1044200030B593B00546222269464FF4002000F0D3
:10443000ABF8222209A94FF4012000F0A5F8684644
:10444000FFF722FF044609A8FFF71EFF54EA000108
:1044500008D07CB118B10A99019888420AD3222267
:10446000694609E022212846FBF7D4FF4FF0FF30D0
:1044700013B030BD222209A92846FBF786FF002091
:10448000F6E730B589B005460C466846FFF7C8FF29
:1044900018B14FF0FF3009B030BD01980695401CAF
:1044A0000190ADF81C4001208DF81E00684600F018
:1044B00015F8F0E710B58AB004466846FFF7B0FF7C
:1044C00018B14FF0FF300AB010BD01988DF81140BF
:1044D000401C0190684600F001F8F4E710B58AB07E
:1044E000014622226846FBF750FF6846FFF7C1FEEF
:1044F000ADF820004FF40024204600F0D9F8222225
:104500006946204600F039F94FF40124204600F0B6
:10451000CFF822226946204600F02FF90AB0002089
:1045200010BD00002DE9F04115000E46044626D0CE
:10453000B5F5807F23D800F039F900281FD1114F3D
:10454000002210213846FEF781FA022000F078F8A8
:10455000204600F003F9002404E0305D00F070F81C
:10456000641CA4B2AC42F8D3012210213846FEF7F5
:104570006DFABDE8F04141F2883000F0DDB8BDE8E9
:10458000F0810000000C01402DE9F0410F4F15466D
:104590000E460446002210213846FEF757FA032043
:1045A00000F04EF8204600F0D9F8002404E000BFE7
:1045B00000F042F83055641CAC42F9D33846BDE8EF
:1045C000F04101221021FEF741BA0000000C014029
:1045D00070B50D4D0446002210212846FEF736FA2C
:1045E0009F2000F02DF800F027F8207000F024F84C
:1045F000607000F021F8A0702846BDE870400122EC
:104600001021FEF723BA0000000C014070B5094DDF
:10461000002210212846FEF719FA052000F010F8B4
:1046200000F00AF80446012210212846FEF70EFA8F
:10463000204670BD000C0140FF2000F001B80000D2
:104640002DE9F0470024DFF86090184F0646254614
:104650004FF40048300601D5012200E00022414617
:104660004846FEF7F3F97006060EFFF7D9FD012262
:1046700008213846FEF7EAF9FFF7D2FD6006040E7E
:1046800020213846FEF7D6F9012801D144F0010473
:10469000002208213846FEF7D9F96D1C082DD9DB18
:1046A0002046BDE8F087000000080140000C0140F2
:1046B00070B5054600F07AF8002816D10B4C0022A0
:1046C00010212046FEF7C2F92020FFF7B9FF284647
:1046D00000F044F8012210212046FEF7B7F9BDE8AA
:1046E000704041F2883000F027B870BD000C0140E6
:1046F0002DE9F041C0B015460F4680464FF4807654
:1047000016E03446A54200D8ACB222466946FFF70F
:104710003BFF224639466846FBF7ECFD18B1002006
:1047200040B0BDE8F08108EB0400804627442D1B13
:10473000002DE6D10120F3E770B50546FEF78CF9B0
:10474000044606E0FEF788F9001BA84201D90120C3
:1047500070BDFFF75BFFC007F4D170BD10B5044614
:10476000C0F30740FFF76CFFC4F30720FFF768FFB3
:10477000E0B2BDE81040FFF763BF2DE9F0411546F8
:104780000F4606460DE0F0B2C0F58074A54200D891
:10479000ACB2224639463046FFF7C4FE26442744D1
:1047A0002D1B002DEFD10120BDE8F08110B541F2A5
:1047B0008830FFF7C1FF08B1012010BD074C00226F
:1047C00010212046FEF742F90620FFF739FF0122AB
:1047D00010212046FEF73AF9002010BD000C0140E0
:1047E0002DE9F04717468A460646002412E000BF2E
:1047F0005AF8240081B24FEA104906EB840088463B
:104800000546FDF785FD50B1A81C4946FDF780FD22
:1048100050B1641CBC42EBDB0120BDE8F08706EB25
:104820008401424605A004E006EB84014A460BA041
:10483000891C00F0B5F80020EFE700003E20D0B45E
:10484000C8EBCAA7B0DC20403078255820286C6F10
:10485000773D307825303458290000003E20D0B410
:10486000C8EBCAA7B0DC20403078255820286869FA
:1048700067683D307825303458290000490050EAF7
:10488000C12018BF04204A0D18BF40F0010040F2BB
:10489000FF72B2EB515F08BF40F00200012808BF71
:1048A00005207047002809DB00F01F02012191401C
:1048B0004009800000F1E020C0F88012704709072D
:1048C000090E002804DB00F1E02080F80014704796
:1048D00000F00F0000F1E02080F8141D7047303820
:1048E0000A2801D2012070470020704730B50C46DD
:1048F0001649C1B00978814226D8FE216846FBF7E7
:10490000DFFC05466423012211A11248FEF7C8FD11
:104910002046FBF71BFD82B2642321460D48FEF7BB
:10492000BFFD642302220CA10A48FEF7B9FDAAB21A
:104930004FF4FA7369460748FEF7B2FD642302227A
:1049400006A10448FEF7ACFD41B030BD14000020C4
:104950005B000000180400205D2000000D0A00002C
:104960000168426811448268C06810440844704776
:1049700070B504464FF6FF7000224AF201050CE0C4
:10498000A35C58400023C60702D085EA500000E02F
:1049900040085B1C082BF6DB521C8A42F0D370BD2A
:1049A0000FB405A110B503AB0420029AFFF79EFFD8
:1049B00010BC5DF814FB00004552524F520000003D
:1049C0000FB405A110B503AB0220029AFFF78EFFCA
:1049D00010BC5DF814FB0000494E464F000000007B
:1049E0000FB405A110B503AB0320029AFFF77EFFB9
:1049F00010BC5DF814FB00005741524E000000004F
:104A0000F8B5FEF767F8FFF7AFF9FEF70BFE2D4894
:104A1000416941F0010141614069002200F001005B
:104A2000009011460D20FEF7C3F80D20FEF7B3F8F5
:104A300026482549002401604FF4E131C0E9011402
:104A40000C26C460C0E904468461C461FEF728FCFA
:104A500008B172B6FEE71D4D1D48403528604FF481
:104A60006120C5E90104EC60C5E90446AC61284653
:104A7000EC61FEF715FC08B172B6FEE715494FF47C
:104A8000806201F58860FEF7BDFC2868C16841F0CE
:104A90001001C1600D48104980300160062141605D
:104AA00040F6FF718160FDF7DDFF08B172B6FEE7E9
:104AB000FFF7FCFB10B109A0FFF772FFFEF7FCFD4A
:104AC0000020F8BD0010024000380140180400200A
:104AD0000048004018000020003000405B424C5D60
:104AE0002057323551363420B3F5CABCBBAFCAA704
:104AF000B0DCA3A10000000010B500290AD008789E
:104B0000002807D005487844FCF71CFD002801D098
:104B1000002010BD0248784410BD0000860100004E
:104B20007E01000010B500290AD00878002807D0BF
:104B300005487844FCF706FD002801D0002010BD90
:104B40000248784410BD0000760100006E010000AC
:104B5000FCF70DB9FCF742BA0000000000000000AD
:104B60000102030406070809000000000102030413
:104B70000000000000000000303132333435363799
:104B80003839414243444546403058003031323391
:104B90003435363738396162636465664030780091
:104BA00004000008000000000000000200010000F6
:104BB00010303132333435363738396162636465E9
:104BC0006678700030313233343536373839414207
:104BD000434445465850000002400000000000A039
:104BE0000000000005400000000000C800000000B8
:104BF0000C4000000000409C000000001940000034
:104C00000020BCBE0000000034400000BFC91B8E65
:104C100000000004B5400000504BCFD06607E2CF43
:104C2000010000006C4100003E8251AADFEEA73473
:104C300001000000D9420000DCB5A0E23A301F9725
:104C4000FFFFFFFFB4450000FD25A0C8E9A3C14F49
:104C5000FFFFFFFFFF3F000000000080000000009A
:104C6000FF3F00000000008000000000B84D000879
:104C700000000020180000006C010008D04D000862
:104C800018000020301B0000880100081C000000F4
:104C900043000000F8FFFFFF0C0000000E000000C2
:104CA0000F0000002E000000100100004300000073
:104CB000F8FFFFFF0040404040404040404041413D
:104CC00041414140404040404040404040404040E1
:104CD000404040404005020202020202020202027B
:104CE0000202020202202020202020202020200278
:104CF0000202020202029090909090901010101008
:104D000010101010101010101010101010101010A3
:104D10000202020202028888888888880808080837
:104D20000808080808080808080808080808080803
:104D3000020202024000000000000000000000002B
:104D40000000000000000000000000000000000063
:104D50000000000000000000000000000000000053
:104D60000000000000000000000000000000000043
:104D70000000000000000000000000000000000033
:104D80000000000000000000000000000000000023
:104D90000000000000000000000000000000000013
:104DA0000000000000000000000000000000000003
:104DB00000000000000000000000000001000000F2
:104DC00010000000000000000024F40001000000BA
:0400000508000131BD
:00000001FF
